:100000001DC036C035C05AC333C032C031C030C045
:100010002FC02EC02DC0B3C398C42AC029C028C089
:1000200027C026C025C024C023C0D7C4A6C4A5C4E9
:10003000A4C4A9C4AAC4ABC4B4C4C9C411241FBEF7
:10004000CFE5D2E0DEBFCDBF10E0A0E6B0E0E0E457
:10005000FAE002C005900D92A036B107D9F710E082
:10006000A0E6B0E001C01D92A43EB107E1F725C1B2
:10007000C7CF841795070CF4CA01681779070CF4E9
:10008000CB01089587B9369A349BFECFF89484B19A
:1000900095B17894089587B9369A349BFECFF89439
:1000A00084B195B17894969587959695879599277B
:1000B000089590E040E050E825E030E887FF02C076
:1000C00064277527880F77FF08C0660F771F6227A0
:1000D00073279F5F983090F303C0660F771FF9CFA7
:1000E000CB0108951F93CF9310919D001E5F109236
:1000F000740010927300C0E0C11788F4EC2FFF2742
:10010000E456FF4F60917300709174008081D1DFDD
:100110009093740080937300CF5FC11778F3EC2F36
:10012000FF27E456FF4F8091730090917400892F50
:1001300099278083CF5FEC2FFF27E456FF4F8091F4
:1001400073008083CF911F9108951F93CF931091D7
:1001500084001C5F60E070E0C0E0C11750F4EC2F39
:10016000FF27ED57FF4F8081A4DFBC01CF5FC11790
:10017000B0F3CB01CF911F910895813011F1999B7C
:100180001DC098991BC090916000923318F49F5F36
:1001900090936000999907C0989B05C0992319F026
:1001A000915090936000923329F0992311F4909329
:1001B0007000089581E080937000F7CF9091600007
:1001C000E9CF90E09093600090937000D8CF982F83
:1001D0004423C9F19093610020E0209362003FE046
:1001E000F89490E0222329F080917000882349F14F
:1001F00092E0662349F090E0222331F039E18091CA
:1002000070008823E1F091E080917D00381708F4B8
:1002100090E08091BD00833008F490E0992319F4B8
:10022000AB98AC98AD98913031F09230F1F4AB9836
:10023000AC9AAD9A1AC0AB9AAC98AD9AF6CF92E050
:10024000E3CF91E0D6CF992369F0809161008823B4
:1002500049F42091620081E0282720936200909366
:100260006100BDCF20916200FACF78940895292FC4
:10027000221F2227221FBC0197FF03C070956195A2
:100280007F4FCB014096869FA001879F500D969F80
:10029000500D1124CA016FE870E0ABD3213019F47E
:1002A000709561957F4FCB0108959C0105960B9742
:1002B00010F420E030E0C9010895CFE5D2E0DEBFC0
:1002C000CDBF82E083BF12BA8FEF81BB18BA8FE334
:1002D00087BB1ABA1BBA85E886B984E485BB8CEF64
:1002E00084BB89E08EBD81EA8FBD1BBC1ABC19BCE2
:1002F00018BC8BE085BD88E183BD89B7806889BF64
:100300008FE289B9549A579A41E060E0862F5FDF07
:10031000C098C198C29A1092E3001092E200109225
:10032000D4001092D300109270001092BC00109272
:10033000DB001092DA001092760010929900109271
:10034000E1001092E0001092810010928000109263
:10035000680010926D001092BD001092BE0081E006
:100360000CDFAA9A1092D50078948091760080FFD5
:1003700009C1AE988091BD008823B9F3AE9A88E197
:1003800090E02CE00FB6F894A89581BD0FBE21BD7A
:100390008091BE00882309F4F3C0AE9880E0EDDEC2
:1003A00080E079DE8093D90087E075DE80937B0062
:1003B00086E071DE80936C0085E06DDE8093DE0068
:1003C00084E069DE8093D60083E065DE80937D0063
:1003D00080919900882309F4D1C08091BD008823C1
:1003E00009F4AA9AE090C3002E2D332720583040FC
:1003F0008091D3009091D400281B390B8FEF2138C6
:10040000380714F421E83FEFC90131DF8C01F09087
:10041000C4002F2D3327205830408091E200909166
:10042000E300281B390B8FEF2138380714F421E83B
:100430003FEFC9011CDFEC01B80117FF04C06627BC
:100440007727601B710BCB01880F991F860F971FB1
:1004500068E572E0681B790B7595679575956795EA
:10046000C69FC001C79F900DD69F900D112468ECC8
:1004700070E0BFD2EB01C801861B970B40E85FEF2D
:100480006FE770E0F6DD9093E1008093E000C00F2D
:10049000D11F40E85FEF6FE770E0CE01EADD909397
:1004A0008100809380008091BD00882309F463C09F
:1004B0008091C700809368008091C80080936D0090
:1004C00060916D0063FF10C08E2D99278058904079
:1004D0009093D4008093D3008F2D9927805890401B
:1004E0009093E3008093E2006078809168008270CE
:1004F00040E06DDE41E85FEF2FE730E0809168007B
:10050000992783FF08C03093E1002093E0003093E7
:1005100081002093800086FF08C05093E100409343
:10052000E000309381002093800080FF08C030936A
:10053000E1002093E000509381004093800085FF0C
:1005400008C05093E1004093E00050938100409335
:10055000800060918000709181008091E000909116
:10056000E10028D08091680080937F0080916D0029
:100570008093DC000DCF80936800A0CFA2D12DCF57
:10058000AE9A0CCFAE9AF6CE882349F025EA91E0D8
:1005900022BF98BF08B600FEFDCF8150C9F708956D
:1005A000CF93C82F882321F084E6EEDFC150E1F716
:1005B000CF910895CF92DF92EF92FF920F931F9306
:1005C000CF93DF93EC017B0180917000882349F089
:1005D000CE01EB01EE24FF24E81AF90AD095C1956B
:1005E000DF4FCE0162DEEC01C7015FDE7C012097A8
:1005F00011F4892B19F088E28093DD008091DE00F0
:10060000482F55279701240F351F8091D600992731
:10061000281B390B6A01C80ED91E40E85FEF6FE74F
:1006200070E0C90126DD805880936A0019BC88BD3E
:1006300080917B00482F55279E01240F351F809104
:100640006C009927281B390B8A01080F191F40E8F5
:100650005FEF6FE770E0C9010CDD805880936700A1
:100660001BBC8ABD91E00735110524F487E5C81647
:10067000D1040CF090E0CD2B39F4EF2829F48091CF
:10068000DD00882309F4982F8091D500813059F03E
:100690008091BD00882309F4982F992311F0969A30
:1006A00004C0969802C090E0F3CFDF91CF911F91E4
:1006B0000F91FF90EF90DF90CF9008951F920F92CF
:1006C0000FB60F9211248F939F93809165008150F4
:1006D00080936500882309F048C080E68093650018
:1006E00090917200992319F091509093720080912B
:1006F000BD00882329F08091BD0081508093BD000A
:100700008091BE00882329F08091BE0081508093A3
:10071000BE008091DD00882329F08091DD008150AA
:100720008093DD009923F1F484E680937200909128
:100730006600992319F0915090936600809176009D
:100740008F5F80937600992399F48CE38093660001
:100750008091DA009091DB0001969093DB0080930A
:10076000DA0006C090916600EECF90917200DACF69
:100770009F918F910F900FBE0F901F9018951F9211
:100780000F920FB60F9211241F932F933F934F9305
:100790005F936F937F938F939F93AF93BF93CF9309
:1007A000EF93FF93CCB1809163009927813091053D
:1007B00009F46AC0823091050CF457C0823091056B
:1007C00009F442C0039709F063C080917E00E82FCE
:1007D000FF27ED57FF4FC0838F5F80937E001091FE
:1007E0006400115010936400112309F051C0ADDC76
:1007F000FC01892B21F480918300813031F082E06B
:100800008093BE001092630043C0412F809184000A
:10081000282F33272E5F3F4FE217F3077CF4DF01C9
:10082000FD01ED57FF4F8081A054BF4F8C934F5F68
:10083000842F9927DC018217930794F3AA9887E005
:100840008093BD00A895DECFC093840083E08093A1
:10085000630082E080937E008C2F8E5F8093640023
:10086000992704964597A4F0CDCF892B89F4C535F7
:1008700079F48091D7009091D800803F910541F4A0
:1008800081E08093630004C0C093830082E0F9CFCD
:100890008C2F99279093D8008093D700FF91EF91E8
:1008A000CF91BF91AF919F918F917F916F915F9108
:1008B0004F913F912F911F910F900FBE0F901F905E
:1008C00018951F9381E080939C0012E080939E0016
:1008D0008091E00080939F00809180008093A00031
:1008E00080916F008093A10080917B008093A20093
:1008F00080916C008093A3008091DE008093A4001F
:100900008091D6008093A500809168008093A60016
:1009100080916D008093A700809176008093A8005D
:10092000912F955F809167008093A90080916A0064
:100930008093AA0090939D00D5DB10939900539A61
:10094000559A8FEF8CB91F9108951F920F920FB691
:100950000F9211242F938F939F93AF93BF93EF9395
:10096000FF9320919900822F9927AA27BB27FC018A
:10097000099798F5EB5EFF4F09948FEF8CB92F5FC5
:10098000209399002AC080EFF9CF85E5F7CF109228
:100990006B0080919D008C5F8093D2002F5F20932D
:1009A000990090916B00E92FFF27E456FF4F80815B
:1009B0008CB99F5F90936B008091D200815080939F
:1009C000D200882351F488E08093990006C01092E9
:1009D00099008FEF8CB955985398FF91EF91BF9183
:1009E000AF919F918F912F910F900FBE0F901F90FD
:1009F000189597FB092E07260AD077FD04D00CD056
:100A000006D000201AF4709561957F4F0895F6F78F
:100A1000909581959F4F0895AA1BBB1B51E107C07C
:100A2000AA1FBB1FA617B70710F0A61BB70B881F7E
:100A3000991F5A95A9F780959095BC01CD0108950D
:00000001FF
